:100000000C94DA020C941E030C941E030C941E0331
:100010000C941E030C941E030C941E030C941E03DC
:100020000C941E030C941E030C94D30D0C94A50E7B
:100030000C941E030C941E030C941E030C941E03BC
:100040000C941E030C94AF220C941E030C941E03FC
:100050000C941E030C94421C0C941E030C941E035F
:100060000C941E030C941E030C941E030C941E038C
:100070000C941E030C941E030C941E030C941E037C
:100080000C941E030C941E030C941E030C941E036C
:100090000C941E030C941E030C941E030C941E035C
:1000A0000C941E030C941E030C941E03120F340FA9
:1000B0002210340F2210790F9C0F2210F10F041020
:1000C000D312D3120213021338135813891489144C
:1000D00063138914131413147A1489148914831460
:1000E0002014201420142014201420142014201470
:1000F0002014201420142014201420142014201460
:1001000032143F1446144D14571475FF01E201597F
:100110000259015D025D015E025E02E2000000F034
:10012000A1F0A2F0A329002B00E300E100E0000011
:10013000001E00140004001D7406014E001F001A6A
:100140000016001B0019012A002000080007000605
:10015000005000280021001500090019004F004B35
:1001600000220017000A0005000000C30023002F32
:100170000000004A0000003E002400300000004D56
:100180000000003B0025001C000B0011000000C215
:1001900000260018000D0010005100490027000C37
:1001A000000E00360052002C002D0012000F003708
:1001B00000007FC1002E0013003300380035004CD2
:1001C000002A0031003400E500E4000000010001D5
:1001D0000001000100010000003A001E022002227E
:1001E00002033001003B001F022102230201000133
:1001F000003C002F0226022F00010001003D0030CC
:100200000227023000010001003E003102350035B6
:1002100002000001003F0001000000010000000199
:1002200000400001000000010000000100410052F8
:100230000051002402000001004200240021001EA1
:1002400000010001004300250022001F00370001CB
:10025000004400260023002000270001004500255F
:10026000022E0231002E004C054600010001000163
:10027000003D0400000050010001000100010000E9
:100280000001000100010001000100010001000166
:1002900000F2000100010001000100F000F1000186
:1002A00000F400010001000100F3000100F500016D
:1002B0000001000100010001000000010001000137
:1002C0000000000100000001000100010000000129
:1002D0000000000100010001000100010000000118
:1002E000000100010001000100AA0001000100015D
:1002F000000100AC00A900B600010001000100AB44
:1003000000A800010001000100010001000100013E
:100310000001000100AE00010001000000E200E267
:1003200000E200E200E200000059000100040001C8
:1003300000E20001005A00010001000100E200E2B9
:10034000005B000800070006000100E2005C0001FD
:100350000009000100010001005D0001000100052D
:1003600000000001005E000100000001000000012B
:10037000005F0001000000010000000100600001BA
:1003800000010001000000010061005F005C0059F5
:100390000062000100620060005D005A006200E23D
:1003A00000570061005E005B006200E200570057EA
:1003B0000057005700570001000100010001000133
:1003C000000100000016034500720067006F004442
:1003D000006F007800200045005A00000016034519
:1003E00000720067006F0044006F00780020004535
:1003F000005A0000000403090409026D0004010012
:10040000A0FA090400000103010100092111010003
:1004100001223F000705810308000A0904010001C9
:1004200003010200092111010001224D000705828C
:100430000308000A09040200010300000009211159
:100440000100012236000705830308000A0904039E
:1004500000010300000009211101000122390007F9
:100460000584031000011201100100000008EDFED8
:10047000071301000102000105010906A10105079A
:1004800019E029E715002501950875018102050885
:1004900019012905950575019102950175039101D1
:1004A0000507190029771500250195787501810246
:1004B000C005010980A101850216010026B7001AB6
:1004C00001002AB700751095018100C0050C0901D3
:1004D000A1018503160100269C021A01002A9C0234
:1004E000751095018100C005010902A1010901A152
:1004F00000050919012905150025019505750181DA
:100500000295017503810105010930093115812525
:100510007F95027508810609381581257F9501753B
:10052000088106050C0A38021581257F950175089A
:100530008106C0C005010906A101050719E029E7E8
:100540001500250195087501810295017508810145
:100550000508190129059505750191029501750395
:1005600091010507190029FF150025FF950675085B
:100570008100C00000000000000000000000010237
:1005800004060A0F17202C3A4A5D71879DB3C7DA1B
:10059000E9F5FCFFFCF5E9DAC7B39D87715D4A3ADE
:1005A0002C20170F0A0604020100000000000000C2
:1005B0000000000011241FBECFEFDAE0DEBFCDBF88
:1005C00004B603FE24C08091FB019091FC01A09130
:1005D000FD01B091FE018730904BA740B04BB9F4BC
:1005E0001092FB011092FC011092FD011092FE018D
:1005F00014BE84B7877F84BF88E10FB6F8948093D8
:100600006000109260000FBEE0E0FFE3099511E08A
:10061000A0E0B1E0ECEEF8E402C005900D92A43346
:10062000B107D9F711E0A4E3B1E001C01D92AB3FDF
:10063000B107E1F70E94170B0C9474240C9400008E
:100640001092B9008AE08093B800089594EA9093DC
:10065000BC009091BC0097FFFCCF9091B900987FAF
:10066000983021F0903111F081E008958093BB0023
:1006700084E88093BC008091BC0087FFFCCF809110
:10068000B900887F883111F0803471F780E00895D7
:1006900084E98093BC008091BC0084FDFCCF089568
:1006A0008093BB0084E88093BC008091BC0087FFEE
:1006B000FCCF9091B900987F81E0983209F480E0F6
:1006C000089584E88093BC008091BC0087FFFCCF34
:1006D0008091BB00089580910101811115C080E4D3
:1006E0000E9426038093010181110CC082E10E94C7
:1006F000500380930101811105C08FEF0E945003C8
:10070000809301010E94480384B1807F84B985B140
:10071000807F85B98AB1837F8AB98BB1837F8BB99A
:100720003E98469808950E942605809301010E94F4
:100730006B0380B38C7080BB81B3836F81BBA5E3F7
:10074000B1E0E3E4F1E08EE08E0F11921D928E1382
:10075000FCCF0C941005BF92CF92DF92EF92FF92E4
:100760000F931F93CF93DF9380910101882379F03A
:10077000809134018F5F80933401811108C00E9401
:10078000260580930101811102C00E94B80405E38F
:1007900011E0C0E0D0E0DD24D39482E0C82EEE2446
:1007A000E394F12CC730D10500F58091010181114E
:1007B00064C080E40E94260380930101811112C06D
:1007C00082E10E9450038093010181110BC0C70197
:1007D0000C2E01C0880F0A94EAF780950E945003FE
:1007E000809301010E94480348C0CA30A1F028F458
:1007F000C83059F0C93061F005C0CC3089F070F0D4
:10080000CD3089F0209A289810C0219A29980DC0DF
:10081000229A2A980AC0239A2B9807C0529A01C09C
:10082000539A5B9802C03E9A469890EA9A95F1F7DF
:100830009FB1799902C082E001C080E091709D254E
:10084000982B7C9902C084E001C080E0892B7D99BF
:1008500002C038E001C030E0832B7E9902C020E165
:1008600001C020E0822B9FB19095991F9927991F75
:100870009295990F907E892B0FC080910101811173
:1008800049C080E40E94260380930101882379F106
:10089000B12C0E9448038B2DF8019081981719F014
:1008A0008083C09200010E946B0321960F5F1F4F4F
:1008B000CE30D10509F076CF80910001882361F117
:1008C000815080930001882339F08FE99FE00197E0
:1008D000F1F700C0000020C0A3E4B1E0E5E3F1E0DF
:1008E000CF01825F91919D938E13FCCF15C083E160
:1008F0000E945003809301018111CACF81E40E94BC
:100900002603809301018111C3CF0E946103B82E99
:10091000B094BFCF80E0C0CF0E94B60481E0DF91E9
:10092000CF911F910F91FF90EF90DF90CF90BF90EC
:100930000895E82FF0E0ED5BFE4F80810895089563
:100940000F931F93CF93DF93C3E4D1E010E00C2FFC
:10095000025F899190E00E94681B180F0C13F9CF79
:10096000812FDF91CF911F910F9108950C949305E2
:1009700056985E9825982D9826982E9827982F9807
:100980008FEF90E0909389008093880090938B0084
:1009900080938A0090938D0080938C00259A2D9AE5
:1009A0002FEF80E792E0215080409040E1F700C0B7
:1009B0000000269A2E9A2FEF80E792E02150804087
:1009C0009040E1F700C00000279A2F9A2FEF80E7B0
:1009D00092E0215080409040E1F700C0000025984F
:1009E0002D982FEF80E792E0215080409040E1F772
:1009F00000C0000026982E982FEF80E792E021504B
:100A000080409040E1F700C0000027982F9856984A
:100A10005E9825982D9826982E9827982F980895B7
:100A200089EA8093800089E08093810024982C9843
:100A30003F988AB18F748AB96E98479A8BB1806B50
:100A40008BB9769A0E94B8040C94920580E2809348
:100A500001018091510181110EC00E94200381E0AB
:100A6000809351012FEF83ED90E32150804090401F
:100A7000E1F700C0000080E40E942603809301019A
:100A800081112EC00E94500380930101811128C062
:100A90000E94500380930101811122C08FE30E94C4
:100AA00050038093010181111BC00E94480380E420
:100AB0000E94260380930101811112C08CE00E94E4
:100AC00050038093010181110BC00E945003809359
:100AD0000101811105C08FE30E9450038093010141
:100AE0000E944803809101010895CF93DF93EC01A8
:100AF000662319F0633059F00DC08A81882321F0F4
:100B000085EE0E94771103C085EE0E943F128A8114
:100B1000811103C080E090E002C08AE091E0DF91A3
:100B2000CF91089508956091BD017091BE018091AB
:100B3000BF019091C0010E94741B56985E98259841
:100B40002D9826982E9827982F98823039F0833048
:100B500041F0813041F4259A2D9A0895269A2E9AD3
:100B60000895279A2F9A089581E0089581E00895C5
:100B70000C94B60508950F931F93CF93DF938C01C8
:100B8000FC01C081D181CE010E94ED19BE010E94FD
:100B90006406EC01B8010E94B805882309F48DC0F1
:100BA000F8018281882309F44AC080915D01811196
:100BB0001FC0C431F0E5DF0709F051C00E94BA053B
:100BC00081E080935D010E940C1C90935C018093F6
:100BD0005B0110925401109256011092550110922F
:100BE00058011092570110925A011092590165C094
:100BF00080915B0190915C010E94181C883C9105DA
:100C000070F480915401E82FF0E0EE0FFF1FEB5AD3
:100C1000FE4FD183C0838F5F809354014EC0C43890
:100C200080E5D80721F0C538D04501F13AC0F80178
:100C30008281882341F01092520182E01EC0C438A4
:100C4000E0E5DE0759F580915201811106C086E288
:100C50000E94771186E20E943F1282E01CC0C438D5
:100C6000F0E5DF0741F3C538D045D9F4F8018281BA
:100C7000882331F01092530180E20E948E121DC031
:100C800080915301811106C087E20E94771187E2AB
:100C90000E943F1280E20E9495120FC0C538D045D5
:100CA00029F381E08093520180935301C801DF91C1
:100CB000CF911F910F910C94B40580E0DF91CF91FB
:100CC0001F910F910895089596E0799FF0011124E6
:100CD00094E5899FE00DF11D1124E60FF11DEE0F43
:100CE000FF1FEB5DFE4F859194910895880F991F2A
:100CF000FC01E356F040859194910895880F991F67
:100D0000FC01E35EFE4F8591949108950F931F932C
:100D1000CF93DF93EC01811520E3920750F5C115C5
:100D200080E2D80708F0C3C0CB3BD10590F4C83AA5
:100D3000D10508F06AC0C53AD10508F05BC0C430DF
:100D4000D10508F0D0C1219709F0CAC101E010E037
:100D50000AC2CF3FD10511F008F0C5C1C03FD1058F
:100D600008F0A2C0CE01805E9109089708F4BBC1CB
:100D7000B7C1C13090E5D90709F4A2C020F5C03150
:100D80008FE4D80770F4C11590E4D90708F094C037
:100D9000C11521E3D20708F0A3C1DD278E01106C35
:100DA000E2C1C115D04509F09BC10E94F4148FEF38
:100DB00094E32CE0815090402040E1F700C0000017
:100DC0000E94671CD0C1C11597E5D90758F4C031FE
:100DD00021E5D20708F01CC1C43180E5D80708F42A
:100DE00075C07EC1CE0190578115904108F078C141
:100DF000DF7073C1C53AD10509F477C1C63AD10590
:100E000009F076C102E810E4AEC1C83AD10509F490
:100E100072C1C93AD10509F471C1CA3AD10509F4C0
:100E200070C1CB3AD10509F46FC1CC3AD10509F4B0
:100E30006EC1CD3AD10509F46DC1C03BD10509F4AD
:100E40006CC1CE3AD10509F46BC1CF3AD10509F492
:100E50006AC1C13BD10509F469C1C23BD10509F49E
:100E600068C1C33BD10509F467C1C43BD10509F48E
:100E700066C1C53BD10509F465C1C63BD10509F47E
:100E800064C1C73BD10509F463C1C83BD10509F46E
:100E900062C1C93BD10509F461C1CA3BD10509F45E
:100EA00060C100E014E45FC18E0110655CC1CE0139
:100EB0009F700E947E0658C1DF708E01106A53C178
:100EC0008091DA0181608093DA014DC10E940C1E8D
:100ED000811102C00E94F21D0E94291E90E0909391
:100EE000FB018093FA01C23080E5D80721F480919C
:100EF000FA01816086C0C43090E5D90721F4809161
:100F0000FA0182607EC0C63020E5D20721F48091CC
:100F1000FA01846076C0C83080E5D80719F4809162
:100F2000FA0127C0CA3090E5D90721F48091FA016F
:100F3000806167C0CC3020E5D20721F48091FA01AE
:100F400080625FC0CE3080E5D80721F48091FA013D
:100F5000806457C0C03190E5D90721F48091FA012F
:100F600080684FC0C23120E5D20729F48091FA0190
:100F70008460886046C0C33080E5D80721F4809142
:100F8000FA018E7F3EC0C53090E5D90721F48091EB
:100F9000FA018D7F36C0C73020E5D20721F4809159
:100FA000FA018B7F2EC0C93080E5D80719F48091F3
:100FB000FA0126C0CB3090E5D90721F48091FA01DF
:100FC0008F7E1FC0CD3020E5D20721F48091FA0139
:100FD0008F7D17C0CF3080E5D80721F48091FA01CA
:100FE0008F7B0FC0C13190E5D90721F48091FA01C0
:100FF0008F7707C0C331D04531F48091FA018B7FE0
:10100000877F8093FA018091FA010E942D1EABC068
:101010008D2F99278F70992781309105D9F49E01E2
:101020002370332702C0880F991F2A95E2F79C6826
:101030008E0144E0000F111F4A95E1F7002713705D
:10104000802B912B53E0CC0FDD1F5A95E1F7C07632
:10105000DD272FC08230910531F4DC2FCC278E01A3
:10106000016F106A80C08330910569F4CE018370EE
:10107000992701E010E002C0000F111F8A95E2F7E6
:10108000C8019C680FC084309105B9F4CE0183700B
:10109000992701E010E002C0000F111F8A95E2F7C6
:1010A000C8019A6823E0CC0FDD1F2A95E1F7C07EC6
:1010B000D7708C010C2B1D2B56C08530910531F457
:1010C000DC2FCC278E01046F106A4DC0069709F003
:1010D0004AC0CF71DD27DC2FCC278E01106243C0C0
:1010E00000E010E040C08E013EC001E810E43BC0CB
:1010F00003E810E438C002EE14E435C009EE14E44D
:1011000032C00AEE14E42FC005EB14E42CC006EB49
:1011100014E429C007EB14E426C00CEC14E423C04B
:101120000DEC14E420C003E815E41DC00AE815E442
:101130001AC002E915E417C004E915E414C001E27D
:1011400016E411C003E216E40EC004E216E40BC07C
:1011500005E216E408C006E216E405C007E216E45C
:1011600002C00AE216E4C801DF91CF911F910F91EE
:10117000089596E0799FF001112494E5899FE00D90
:10118000F11D1124E60FF11DEE0FFF1FEB5DFE4F69
:1011900085919491803E9105E0F4803C910558F54D
:1011A0008133910509F46FC048F48932910509F43F
:1011B00063C08A32910509F46DC072C0893391050C
:1011C000E9F082389105D1F08533910509F44DC0DD
:1011D00067C0833E910581F138F4803E9105B9F0F6
:1011E000823E9105D9F05CC0863E910561F1873E53
:1011F0009105A1F155C00E94760608952091FA014B
:1012000020FD02C021FF4CC080EE90E049C08091DB
:10121000FA0180FFF9CF89E390E042C08091FA01A2
:1012200082FF0EC08091FA0184FF03C080E090E04D
:1012300037C083EE90E034C08091FA0182FFF2CF94
:1012400082EE90E02DC08091FA0183FF0BC0809167
:10125000FA0184FDEBCF87EE90E022C08091FA0185
:1012600083FFF5CF86EE90E01BC08091FA0185FFE9
:1012700007C089E290E014C08091FA0185FFF9CFA0
:1012800085E390E00DC08091FA0186FF07C08AE2F5
:1012900090E006C08091FA0186FFF9CF81E390E0EB
:1012A0000E948606089508950C94530980916E015A
:1012B0000895CF93DF9300D01F92CDB7DEB79C0186
:1012C0008091F101843019F593E099833B832A835F
:1012D0009093E9008FEF9091E800815095FD06C052
:1012E00095ED9A95F1F700008111F5CF8091E80016
:1012F00085FF0DC040E050E063E070E0CE01019654
:101300000E94C30B8091E8008E778093E8000F90D5
:101310000F900F90DF91CF910895CF93DF9300D07E
:101320001F92CDB7DEB72091F101243021F522E0E4
:1013300029839B838A8383E08093E9008FEF9091D8
:10134000E800815095FD06C095ED9A95F1F70000F3
:101350008111F5CF8091E80085FF0DC040E050E09D
:1013600063E070E0CE0101960E94C30B8091E8001B
:101370008E778093E8000F900F900F90DF91CF91C0
:1013800008952091F1012430F1F422E02093E90046
:101390002FEF3091E800215035FD06C035ED3A952C
:1013A000F1F700002111F5CF2091E80025FF0BC0D7
:1013B00040E050E065E070E00E94C30B8091E800DF
:1013C0008E778093E8000895CF93DF93EC0190919E
:1013D000F101943009F046C080910C018823D9F0C6
:1013E00080910D018823B9F09093E9008FEF9091DF
:1013F000E800815095FD06C095E19A95F1F700004F
:101400008111F5CF8091E80085FF2CC040E050E0CD
:1014100060E170E017C081E08093E9008FEF909168
:10142000E800815095FD06C095ED9A95F1F7000012
:101430008111F5CF8091E80085FF14C040E050E0B5
:1014400068E070E0CE010E94C30B8091E8008E77C7
:101450008093E80080E1FE01AEE5B1E001900D92DD
:101460008A95E1F7DF91CF9108958091F001811184
:1014700009C00E94580D0E94B50D8091E200846061
:101480008093E20008951092F001089508950C945D
:101490009C220E94FD1B0E94A2220E945B100C94C1
:1014A000540942E061EC81E00E94D20C42E061EC20
:1014B00082E00E94D20C42E061EC83E00E94D20CF8
:1014C00042E161EC84E00C94D20C8091F301833012
:1014D00009F455C030F4813071F0823009F48EC0C7
:1014E00008958A3009F47AC08B3009F460C08930DD
:1014F00009F09CC020C08091F201813A09F096C0A9
:101500008091E800877F8093E8008091F6019091B8
:10151000F701892B21F460E18EE591E003C060E0E2
:1015200080E090E070E00E940E0C8091E8008B77E4
:101530008093E80008958091F201813209F076C02D
:101540008091F6019091F701009719F0039709F047
:101550006DC08091E800877F8093E8008091E8006B
:1015600082FD05C08091F1018111F8CF5FC08091AB
:10157000F10080936E018091E8008B7753C08091D9
:10158000F201813A09F052C08091F6019091F70181
:10159000892B09F04BC08091E800877F8093E80099
:1015A0008091E80080FFFCCF80910C0136C08091D3
:1015B000F2018132D9F58091F6019091F701892BE2
:1015C000A9F58091E800877F8093E8000E94070DCD
:1015D0008091F40180930C010C94F4148091F20139
:1015E000813221F58091E800877F8093E8000E9496
:1015F000070D8091F50180936F0108958091F201AC
:10160000813AA1F48091E800877F8093E80080917F
:10161000E80080FFFCCF80916F018093F100809102
:10162000E8008E778093E8000C94070D089584B746
:10163000877F84BF88E10FB6F89480936000109292
:1016400060000FBE90E080E80FB6F89480936100D0
:10165000909361000FBE0E94AA100E94580D0E9434
:10166000B50D8091E20084608093E20078940E943E
:101670003B100E94AC1082E091E00E9456100E9444
:101680008A228091F101853069F40E94C41B809107
:10169000EF018823B1F30E94EF1B882391F30E948E
:1016A000AD0BEFCF0E94B210ECCF292F33272330A0
:1016B0003105C9F064F42130310581F02230310563
:1016C00009F043C08DE690E029EF33E042C02132BB
:1016D0003105F1F02232310541F137C082E190E06D
:1016E00026E634E036C099278130910541F08230FA
:1016F000910541F0892B49F5E5EFF3E005C0EDEDEB
:10170000F3E002C0E5ECF3E0849190E09F0121C09A
:101710006430D8F4E62FF0E0EE0FFF1FEE5DFE4FD1
:101720002081318189E090E014C0643070F470E071
:10173000FB01EE0FFF1FE65EFE4F20813181FB01B2
:10174000EA5EFE4F808190E004C080E090E020E0FF
:1017500030E0FA0131832083089580E189BD82E180
:1017600089BD09B400FEFDCF8091D8008F7D8093A4
:10177000D8008091E00082608093E0008091E000DA
:1017800081FDFCCF0895CF92DF92EF92FF920F93ED
:101790001F93CF93DF93EC018B016A010E94260D0A
:1017A000811133C0C114D10439F0F60180819181D7
:1017B000081B190BC80FD91FE12CF12C01151105BD
:1017C00019F18091E80085FD16C08091E8008E77C0
:1017D0008093E800C114D10449F0F6018081918121
:1017E000E80EF91EF182E08285E00FC00E94260D0E
:1017F000882321F30AC089918093F10001501109D7
:10180000FFEFEF1AFF0ADACF80E0DF91CF911F914F
:101810000F91FF90EF90DF90CF9008952091F80105
:101820003091F9012617370748F06115710539F431
:101830002091E8002E772093E80001C0B90140E034
:1018400061157105A9F12091F101222309F443C02A
:10185000253009F442C02091E80023FD40C02091CA
:10186000E80022FD32C02091E80020FFE9CF40913E
:10187000F3002091F20030E0342BFC01CF01611520
:10188000710559F02830310540F481918093F100C1
:10189000615071092F5F3F4FF1CF41E02830310592
:1018A00009F040E02091E8002E772093E800C8CFAF
:1018B0004111C9CF0AC08091F101882361F08530C0
:1018C00061F08091E80083FD0AC08091E80082FF0A
:1018D000F2CF80E0089582E0089583E0089581E0EA
:1018E00008952091F8013091F9012617370748F043
:1018F0006115710539F42091E8002E772093E800F6
:1019000001C0B901FC0120E06115710591F18091E0
:10191000F101882309F440C0853009F43FC080916B
:10192000E80083FD3DC08091E80082FD2FC08091DA
:10193000E80080FFE9CF2091F3008091F20090E071
:10194000922B6115710559F08830910540F424916E
:101950002093F1003196615071090196F2CF21E098
:10196000089709F020E08091E8008E778093E800E6
:10197000CBCF2111CCCF0AC08091F101882361F037
:10198000853061F08091E80083FD0AC08091E80015
:1019900082FFF2CF80E0089582E0089583E0089509
:1019A00081E00895982F973058F59093E9009817A3
:1019B00039F07091EC002091ED005091F00003C0DF
:1019C000242F762F50E021FF19C03091EB003E7F8D
:1019D0003093EB003091ED003D7F3093ED0030917E
:1019E000EB0031603093EB007093EC002093ED003E
:1019F0005093F0002091EE0027FF07C09F5FD3CFE8
:101A00008F708093E90081E0089580E008958091CF
:101A1000F20187FF11C08091E80082FD05C080912E
:101A2000F1018111F8CF11C08091E8008B770BC0D4
:101A30008091F101882349F08091E80080FFF8CF80
:101A40008091E8008E778093E80008952091E4006B
:101A50003091E50095E64091EC00842F817040FFC5
:101A600022C08091E80080FD1CC08091F101882394
:101A700091F0853091F08091EB0085FD10C0409190
:101A8000E4005091E5004217530729F39A01915061
:101A900011F784E0089582E0089583E0089581E0DD
:101AA000089580E008954091E80042FFDECF089558
:101AB0000E94C60D0E94CE0DE0EEF0E080818160B4
:101AC0008083E8EDF0E080818F77808319BCA7EDFB
:101AD000B0E08C918E7F8C9380818F7E808310927A
:101AE000F00108950F931F93CF93DF930E94C60DCB
:101AF0000E94CE0DC8EDD0E088818F7788838881E1
:101B00008068888388818F7D888319BC1092F10159
:101B10001092ED011092EF011092EE0100EE10E034
:101B2000F80180818B7F808388818160888342E097
:101B300060E080E00E94D20CE1EEF0E080818E7FD8
:101B40008083E2EEF0E08081816080838081886024
:101B50008083F80180818E7F808388818061888383
:101B6000DF91CF911F910F910895E8EDF0E0808112
:101B70008F7E8083E7EDF0E080818160808384E068
:101B800082BF81E08093F0010C94720DE8EDF0E0EB
:101B900080818E7F80831092E20008951092DA0097
:101BA0001092E10008951F920F920FB60F92112428
:101BB0002F933F934F935F936F937F938F939F9355
:101BC000AF93BF93EF93FF938091E10082FF0BC02F
:101BD0008091E20082FF07C08091E1008B7F8093BB
:101BE000E1000E943A108091DA0080FF1FC08091CE
:101BF000D80080FF1BC08091DA008E7F8093DA00CE
:101C00008091D90080FF0DC080E189BD82E189BD4E
:101C100009B400FEFDCF81E08093F1010E94350AF6
:101C200005C019BC1092F1010E94430A8091E100A5
:101C300080FF19C08091E20080FF15C08091E20012
:101C40008E7F8093E2008091E20080618093E200C9
:101C50008091D80080628093D80019BC85E0809381
:101C6000F1010E94470A8091E10084FF30C0809119
:101C7000E20084FF2CC080E189BD82E189BD09B406
:101C800000FEFDCF8091D8008F7D8093D800809199
:101C9000E1008F7E8093E1008091E2008F7E80934F
:101CA000E2008091E20081608093E2008091ED018A
:101CB000882311F084E007C08091E30087FD02C013
:101CC00081E001C083E08093F1010E94490A809184
:101CD000E10083FF29C08091E20083FF25C080914D
:101CE000E100877F8093E10082E08093F101109210
:101CF000ED018091E1008E7F8093E1008091E20010
:101D00008E7F8093E2008091E20080618093E20008
:101D100042E060E080E00E94D20C8091F000886098
:101D20008093F0000E94460AFF91EF91BF91AF911E
:101D30009F918F917F916F915F914F913F912F91E3
:101D40000F900FBE0F901F9018951F920F920FB615
:101D50000F9211242F933F934F935F936F937F9331
:101D60008F939F93AF93BF93CF93DF93EF93FF93A3
:101D7000C091E900CF708091EC00D82FD17080FD28
:101D8000D0E81092E9008091F000877F8093F00006
:101D900078940E94E90E1092E9008091F00088602A
:101DA0008093F000CD2BCF70C093E900FF91EF91AD
:101DB000DF91CF91BF91AF919F918F917F916F9163
:101DC0005F914F913F912F910F900FBE0F901F90F9
:101DD00018951F93CF93DF93CDB7DEB7AA970FB6B1
:101DE000F894DEBF0FBECDBFE2EFF1E088E08E0FCA
:101DF0009091F10091938E13FBCF0E94650A809120
:101E0000E80083FF1FC18091F2019091F301492FF7
:101E100050E04A30510508F015C1FA01EA5AFF4F67
:101E20000C942424803881F0823809F00BC1809111
:101E3000F6018F708093E9008091EB0085FB882785
:101E400080F91092E90006C08091EE019091EF01B7
:101E5000911182609091E800977F9093E8008093C1
:101E6000F1001092F100C8C0282F2D7F09F0EAC0C0
:101E7000882319F0823061F0E5C08091F40181304F
:101E800009F0E0C0933009F080E08093EF012BC0AF
:101E90008091F401811127C08091F6018F7009F4BF
:101EA000D1C08093E9002091EB0020FF1CC093304B
:101EB00021F48091EB00806214C09091EB0090615E
:101EC0009093EB0021E030E0A90102C0440F551FC0
:101ED0008A95E2F74093EA001092EA008091EB00C5
:101EE00088608093EB001092E9008091E800877F82
:101EF00086C08111A7C01091F4011F778091E30083
:101F00008078812B8093E3008091E800877F809325
:101F1000E8000E94070D8091E80080FFFCCF8091CF
:101F2000E30080688093E300111102C082E001C0E9
:101F300083E08093F10186C08058823008F082C02F
:101F40008091F4019091F5018C3D53E0950779F56E
:101F500083E08A838AE289834FB7F894DE0113967F
:101F600020E03EE051E2E32FF0E050935700E4918F
:101F700020FF03C0E295EF703F5FEF708E2F90E07F
:101F8000EA3010F0C79601C0C0968D939D932F5FE5
:101F9000243149F74FBF8091E800877F8093E800A4
:101FA0006AE270E0CE0101960E940E0C14C0AE01F0
:101FB0004F5F5F4F6091F6010E94550BBC01009787
:101FC00009F440C09091E800977F9093E8008981E0
:101FD0009A810E94710C8091E8008B778093E800D1
:101FE00031C0803879F58091E800877F8093E800E0
:101FF0008091ED018093F1008091E8008E778093CD
:10200000E8000E94070D1EC081111CC09091F401D0
:102010009230C0F48091E800877F8093E80090932D
:10202000ED010E94070D8091ED01811106C08091A4
:10203000E30087FD02C081E001C084E08093F101EC
:102040000E94510A8091E80083FF0AC08091E80055
:10205000877F8093E8008091EB0080628093EB00A3
:10206000AA960FB6F894DEBF0FBECDBFDF91CF9119
:102070001F9108950895CF938091F1018823A1F0D5
:10208000C091E900CF709091EC00892F817090FD94
:1020900080E8C82B1092E9008091E80083FD0E943F
:1020A000E90ECF70C093E900CF9108959093750128
:1020B000809374010895E0917401F0917501309757
:1020C00021F00190F081E02D099480E00895E091E5
:1020D0007401F0917501309721F00280F381E02DB9
:1020E00009940895E0917401F0917501309721F001
:1020F0000480F581E02D09940895209172013091BA
:1021000073018217930771F09093730180937201AA
:10211000E0917401F0917501309721F00680F7810C
:10212000E02D09940895209170013091710182177A
:10213000930771F09093710180937001E0917401A5
:10214000F0917501309721F00084F185E02D09941C
:10215000089508950C94A9100E94031C0E949303F3
:102160000C94C51C9F92AF92BF92CF92DF92EF92D8
:10217000FF920F931F93CF93DF9300D000D000D036
:10218000CDB7DEB70E94AB030DE010E0AA24A39404
:10219000B12C902E802F0E949904980129583E4F0F
:1021A0006901F901F080F826A1F40150110988F7BE
:1021B0008FEF89838A831B820E940C1C8160782F99
:1021C0009D838C8349815A816B818D810E94491145
:1021D0002FC09091DA0191FF04C08E830E949F046A
:1021E0008E8125E030E0A501022E01C0440F0A9443
:1021F000EAF7E42E4F21C1F029839A828E2191E0E3
:1022000009F490E09B830E940C1C8160782F9D83D1
:102210008C8349815A816B818D810E944911F6011D
:102220008081E826E08204C021503109E0F6BDCF6C
:102230000E94AC1F109176010E945B101817B9F034
:102240000E945B108093760126960FB6F894DEBF4D
:102250000FBECDBFDF91CF911F910F91FF90EF90F7
:10226000DF90CF90BF90AF909F900C94540926962A
:102270000FB6F894DEBF0FBECDBFDF91CF911F9197
:102280000F91FF90EF90DF90CF90BF90AF909F9015
:102290000895CF93DF93CDB7DEB72B970FB6F894A1
:1022A000DEBF0FBECDBF4F83588769877A878B8784
:1022B000DE01119686E0FD0111928A95E9F785E02D
:1022C000FE01379601900D928A95E1F749815A8176
:1022D0006B817C818D819E810E9492172B960FB617
:1022E000F894DEBF0FBECDBFDF91CF910895CF939D
:1022F000882309F4C2C0C82F823859F40E945B10A9
:1023000081FDBBC089E30E946C1A0E94391B89E3DE
:102310000CC0833879F40E945B1080FDAEC083E569
:102320000E946C1A0E94391B83E50E94AE1ACF915D
:102330000C94391B843859F40E945B1082FD9DC0B7
:1023400087E40E946C1A0E94391B87E4EECF8CEF61
:102350008C0F813A48F48C2F0E94EF2181118DC09F
:102360008C2F0E946C1AE3CF80E28C0F883048F4E7
:10237000C77081E001C0880FCA95EAF70E94F21A7F
:10238000D6CF8BE58C0F833078F4C53A29F0C63A66
:1023900031F083E890E005C081E890E002C082E877
:1023A00090E0CF910C947D1088E58C0F833108F07C
:1023B00064C0C83A39F1C93A41F1CA3A49F1CB3A55
:1023C00051F1CC3A59F1CD3A61F1C03B69F1CE3AC5
:1023D00071F1CF3A79F1C13B81F1C23B89F1C33B45
:1023E00091F1C43B99F1C53BA1F1C63BA9F1C73BB3
:1023F000B1F1C83BB9F1C93BC1F1CA3BC9F180E0B9
:1024000090E038C082EE90E035C089EE90E032C0B6
:102410008AEE90E02FC085EB90E02CC086EB90E038
:1024200029C087EB90E026C08CEC90E023C08DECB7
:1024300090E020C083E891E01DC08AE891E01AC0D6
:1024400082E991E017C084E991E014C081E292E052
:1024500011C083E292E00EC084E292E00BC085E2FC
:1024600092E008C086E292E005C087E292E002C0F6
:102470008AE292E0CF910C949310CF910895882333
:1024800009F44BC0823859F40E945B1081FF45C0AB
:1024900089E30E946C1A0E94391B89E30CC08338BF
:1024A00071F40E945B1080FF38C083E50E946C1AB3
:1024B0000E94391B83E50E94AE1A0C94391B8438A4
:1024C00059F40E945B1082FF28C087E40E946C1AB6
:1024D0000E94391B87E4EFCF9CEF980F913A58F395
:1024E00090E2980F983050F4877091E001C0990FF6
:1024F0008A95EAF7892F0E94F81ADFCF9BE5980F9B
:10250000933020F480E090E00C947D10885A833161
:1025100020F480E090E00C9493100895882321F03B
:102520000E94F21A0C94391B0895882321F00E940E
:10253000F81A0C94391B08957F928F929F92AF9254
:10254000BF92CF92DF92EF92FF920F931F93CF93A0
:10255000DF931F92CDB7DEB77C01C62E772EFC012C
:10256000058102950F70128111110E940F1B0E94AC
:10257000651A882379F0112369F080E28C0D883088
:1025800048F082E00E944E1A0E94651A91E0D82E0F
:10259000D92601C0D12CE72DE295EF70F0E0E05A8A
:1025A000FF4F0C942424872D807F072D0F708823E4
:1025B00011F00295007F112389F0002309F490C1E6
:1025C00080E28C0D883020F4802F0E94F21A03C024
:1025D000802F0E94021B0E94391B82C18C2D0E94F9
:1025E0003F12002309F495C180E28C0D883020F45D
:1025F000802F0E94F81A03C0802F0E94081B0E949F
:10260000391B87C1972D907F872D8F70903211F0E5
:102610008295807FCC2021F0F1E0CF16B1F01EC072
:10262000112349F0002309F414C1013009F011C14C
:102630000E94221B6EC1002319F0013009F469C108
:1026400089830E94251B89810AC1112321F0023050
:1026500008F05FC1FEC001115CC101C1112321F06E
:10266000002309F4F6C03CC1002309F4F8C03EC1C0
:10267000872D86958695837090E0009719F00197D5
:1026800061F047C1112321F08C2D972D937002C06A
:1026900080E090E00E947D103CC1112321F08C2D40
:1026A000972D937002C080E090E00E94931031C19A
:1026B0008C2D112319F00E94B41E02C00E941C1F11
:1026C0000E94A11F26C1872D837009F052C01111ED
:1026D00020C18C2D829586958770880F880F9C2D40
:1026E0009F70892E912CA12CB12C082E04C0880C2F
:1026F000991CAA1CBB1C0A94D2F7C4FE14C00FE09C
:1027000010E020E030E0B901A80104C0440F551FDB
:10271000661F771F8A95D2F7CB01BA016095709535
:102720008095909503C060E070E0CB01272D269541
:102730002695237030E02230310569F023303105D1
:1027400089F0682979298A299B292130310571F07E
:102750000E94DA18DEC0682979298A299B290E94FB
:10276000F618D7C00E94DA18C501B4010E94BE183D
:10277000D0C0112319F0872D817001C08695882360
:1027800009F4C7C08C2D829586958770880F880FB5
:102790009C2D9F70892E912CA12CB12C082E04C049
:1027A000880C991CAA1CBB1C0A94D2F7C4FE14C046
:1027B0000FE010E020E030E0B901A80104C0440FB0
:1027C000551F661F771F8A95D2F7CB01BA01609516
:1027D00070958095909503C060E070E0CB01272D47
:1027E000269526952370422F50E04230510569F01E
:1027F0004330510589F0682979298A299B2941307C
:10280000510571F00E94B41984C0682979298A2978
:102810009B290E94D0197DC00E94B419C501B40142
:102820000E94981976C08C2D90E0FC01E05EF109C1
:10283000E531F10508F050C0E059FF4F0C94242415
:102840000C2D0F70872D8F71112331F00E943119DB
:10285000802F0E948E125DC00E945219802F0E940C
:10286000951257C0112339F0011153C0872D8F7174
:102870000E9477194EC0023008F04BC0F7CF1123E9
:1028800039F0872D8F710E94311943C01123C9F38C
:10289000872D8F710E9452193CC0112329F0872D7A
:1028A0008F710E941C1935C00E94121932C0112369
:1028B00051F0172D1F71812F0E94311963E0812F74
:1028C0000E94451A26C081E00E944E1A023008F18B
:1028D00082E00E944E1A1DC0112331F0002389F2BC
:1028E0008C2D0E94771115C0002391F28C2D0E942F
:1028F0003F120FC0472D4F706C2DC7010E94750508
:102900000E94361806C0472D4F706C2DC7010E94DB
:102910006306DD20F9F00E94411A80FD1BC0F7011B
:1029200012820E943B1A0E943119C7010E94B914F9
:102930000E943B1A0F90DF91CF911F910F91FF9052
:10294000EF90DF90CF90BF90AF909F908F907F904F
:102950000C9452190F90DF91CF911F910F91FF901E
:10296000EF90DF90CF90BF90AF909F908F907F902F
:1029700008950F931F93CF93DF93EC018881998182
:102980002B813C81232BB9F09F3F11F48F3F99F0AD
:10299000CE010E94BB05882371F0688179818A810C
:1029A0000E94371A8C010E94EC190E94B318B801DA
:1029B000CE010E949C12DF91CF911F910F9108953B
:1029C0000E940F1B0E941F1B0E94E41A0E94391BC9
:1029D0000E9452200E94A11F80E090E00E947D1082
:1029E00080E090E00C9493100E94FF1A0C94E01485
:1029F0000E942C1A292F22952F7030E02C3031059F
:102A00004CF42A3031056CF4225031092230310562
:102A1000A8F407C02C30310569F02F30310551F092
:102A20000DC0803F69F018F4803E40F409C0843F37
:102A300029F406C093FB882780F9089580E0089563
:102A400081E00895CF93DF9300D000D01F92CDB7DF
:102A5000DEB70F900F900F900F900F90DF91CF91F6
:102A60000895CF93DF9300D000D000D0CDB7DEB76C
:102A700026960FB6F894DEBF0FBECDBFDF91CF9183
:102A800008951F93CF93DF93C091850116E0809145
:102A90008601C81799F0D0E01C9FF0011D9FF00D32
:102AA0001124E957FE4F40815181628173818481F5
:102AB00095810E9431152196C770E9CFDF91CF91A2
:102AC0001F9108954091B7015091B8016091B901EB
:102AD0007091BA018091BB019091BC010C943115A9
:102AE0008091BC0182958F7009F054C08091B9012A
:102AF000882309F44FC080918501A09186016091DF
:102B0000B7017091B8014091BA015091BB01B6E094
:102B10008A1709F43FC090E041155105C1F17F3F8C
:102B200011F46F3FA1F1B89FF001B99FF00D11248E
:102B3000E957FE4F218172132AC02081621327C0FA
:102B40002281211124C0238134812417350710F4F8
:102B500021503109241B350B283C3105C0F420914C
:102B6000BC012F7020612093BC0126E0289FF0015A
:102B7000299FF00D1124E457FE4F80818F708061F2
:102B8000808387EB91E00E94B9140C944115019663
:102B90008770BECF0895CF92DF92EF92FF920F938E
:102BA0001F93CF93DF93CDB7DEB762970FB6F8943C
:102BB000DEBF0FBECDBF8C0185E0F801DE011D96A2
:102BC00001900D928A95E1F7D8014C9111965C9194
:102BD000119712966C9112971396CD90DC901497E2
:102BE0003091B7017091B8018091BA019091BB0109
:102BF000009709F46BC17F3F19F43F3F09F466C1A8
:102C0000E090B901EE2009F4C0C02091BC01C816C3
:102C1000D90628F0F601E81BF90BCF0104C0809516
:102C200090958C0D9D1DFF24F394883C910578F0C0
:102C3000F12C207F09F0C6C07C2DD98AC88A8989E9
:102C40000E94221587EB91E00E94B914B1C0822F37
:102C5000807F09F046C0751314C0341312C061118F
:102C600010C02F7020612093BC010E94621587EB79
:102C700091E00E94B9148091BC01D80115968C9303
:102C80002EC0CD2819F15F3F11F44F3FF9F0F62E19
:102C900061111CC0809185012091860136E0821768
:102CA00009F45AC090E0389FF001399FF00D1124CB
:102CB000E957FE4F7181571306C07081471303C057
:102CC0007281711103C001968770E9CFF62E6623D9
:102CD00009F418C18091BC0181608093BC01F12C82
:102CE00011C1751308C0341306C0611104C080916E
:102CF000BC01D801C3C04D875E878D859E856A8BD8
:102D00000E94F8146A898823E1F16623D1F12091A9
:102D1000BC01822F82958F7090E0029774F08091B1
:102D2000B7019091B80198878F831986DB86CA8690
:102D30002C87CE0107960E94B91486E0F801A7EB14
:102D4000B1E001900D928A95E1F70E9470150E9402
:102D50006215FF24F394D6C04D875E878D859E85CE
:102D60000E942C1A292F22952F7030E02230310535
:102D70000CF0BCC09F7009F0B6C0805E883008F4CB
:102D8000C1C0C8010E94B914E4CFC816D90608F41E
:102D900053C0F601E81BF90BCF01883C910508F4FC
:102DA00050C0F12C7C2DD98AC88A89890E942215AD
:102DB000E7EBF1E086E0DF011D928A95E9F70E94DA
:102DC0006215A0C0751314C0341312C0611110C075
:102DD0008091BC01F8018583C8010E94B91486E086
:102DE000E7EBF1E0DF011D928A95E9F7FE2C8AC03E
:102DF0004D875E878D859E856A8B0E94F8146A894F
:102E0000882309F4BECF662309F4BBCF2091BC010F
:102E1000822F82958F7090E002970CF48ECF809174
:102E2000B7019091B8019A8389831B82DD82CC829D
:102E30002E83CE0101967FCF809590958C0D9D1DA0
:102E4000ACCFF62E662309F49CCF75132EC0341335
:102E50002CC02091BC0120FD1FC0822F82958F7055
:102E6000D9F0D80115962C9315978F3049F08F5FC4
:102E7000982F9295907F822F8F70892B15968C9327
:102E8000C8010E94B91486E0F801A7EBB1E00190F7
:102E90000D928A95E1F793CF86E0F801A7EBB1E0B8
:102EA00001900D928A95E1F72DC04D875E878D8543
:102EB0009E850E94F814811140CF8091BC018160F1
:102EC0008093BC01C8010E94B9141CC0662309F498
:102ED00058CF4D875E878D859E850E94F814882384
:102EE00009F44FCF2ACF811148CF0CC024303105CF
:102EF0000CF047CF9F7009F440CFF8019581907F87
:102F000009F03BCF8F2D62960FB6F894DEBF0FBE4F
:102F1000CDBFDF91CF911F910F91FF90EF90DF9088
:102F2000CF9008951F93CF93DF93CDB7DEB72C9743
:102F30000FB6F894DEBF0FBECDBF4F8358876987A9
:102F40007A878B879C87CE0107960E94CB158823B2
:102F500069F08F8198852A853B85232BF1F19F3F6E
:102F600009F063C08F3F09F060C037C086E0FE0102
:102F70003796DE01119601900D928A95E1F76F81E7
:102F80007885EA85FB85309741F17F3F11F46F3FEB
:102F900021F12091860130E0C901019687709927BF
:102FA0004091850150E08417950709F447C0698373
:102FB0007A83FD83EC8396E0929FD001939FB00DBE
:102FC0001124A957BE4FFE01319601900D929A959A
:102FD000E1F7809386010E94411516E080918501FA
:102FE000909186018917C1F1189FC001112489575A
:102FF0009E4F0E94CB15882379F1E09185011E9F99
:10300000F0011124E957FE4F4081518162817381A3
:10301000848195810E9431158091850190E001960F
:103020008770992780938501D9CF4F81588569850D
:103030007A858B859C850E943115CFCF0E94F41430
:103040001092860110928501E7EBF1E086E0DF0146
:103050001D928A95E9F7C1CF2C960FB6F894DEBF82
:103060000FBECDBFDF91CF911F910895EF92FF92D8
:103070000F931F93CF93DF938C01009709F46CC0DB
:10308000F12CEE24E394E8012196F8018491843731
:1030900040F4843008F051C0813081F0823019F161
:1030A0005BC0853709F444C0A8F19CE7980F9037BE
:1030B00008F052C08F770E943F1241C00E5F1F4F31
:1030C000FE01C49180E28C0F883048F4C7708E2DC9
:1030D00001C0880FCA95EAF70E94121B14C08C2FFA
:1030E0000E9477112DC00E5F1F4FFE01C49180E238
:1030F0008C0F883058F4C7708E2D01C0880FCA9588
:10310000EAF70E94181B0E94391B1AC08C2F0E94DC
:103110003F1216C00E5F1F4FFE01C491CC2381F0F9
:103120008FE99FE00197F1F700C00000C150F6CF92
:103130000E5F1F4FFE01F49003C00E9477118E01B5
:103140008F2D882309F49FCFEFE9FFE03197F1F746
:1031500000C000008150F5CFDF91CF911F910F91FA
:10316000FF90EF90089508956093C1017093C2019C
:103170008093C3019093C4010C94E0140F931F93A8
:103180000091C1011091C2012091C3013091C4018D
:10319000DC01CB01802B912BA22BB32B8093C1019F
:1031A0009093C201A093C301B093C4011F910F91EA
:1031B0000C94E0140F931F930091C1011091C20170
:1031C0002091C3013091C401DC01CB018023912304
:1031D000A223B3238093C1019093C201A093C301A2
:1031E000B093C4011F910F910C94E0140F931F939F
:1031F0000091C1011091C2012091C3013091C4011D
:10320000DC01CB0180279127A227B3278093C1013E
:103210009093C201A093C301B093C4011F910F9179
:103220000C94E0141092BD011092BE011092BF01E7
:103230001092C0010C94E01441E050E060E070E0B6
:1032400004C0440F551F661F771F8A95D2F740931D
:10325000BD015093BE016093BF017093C0010C94F7
:10326000E01441E050E060E070E004C0440F551FFE
:10327000661F771F8A95D2F78091BD019091BE019C
:10328000A091BF01B091C001482B592B6A2B7B2B19
:103290004093BD015093BE016093BF017093C00184
:1032A0000C94E01441E050E060E070E004C0440F92
:1032B000551F661F771F8A95D2F7409550956095E8
:1032C00070958091BD019091BE01A091BF01B09118
:1032D000C001482359236A237B234093BD015093A7
:1032E000BE016093BF017093C0010C94E01441E0F3
:1032F00050E060E070E004C0440F551F661F771F68
:103300008A95D2F78091BD019091BE01A091BF0135
:10331000B091C001482759276A277B274093BD01F8
:103320005093BE016093BF017093C0010C94E014F0
:103330000F931F930091BD011091BE012091BF0119
:103340003091C001DC01CB01802B912BA22BB32B40
:103350008093BD019093BE01A093BF01B093C001C3
:103360001F910F910C94E0140F931F930091BD01D6
:103370001091BE012091BF013091C001DC01CB0151
:1033800080239123A223B3238093BD019093BE0198
:10339000A093BF01B093C0011F910F910C94E01452
:1033A0000F931F930091BD011091BE012091BF01A9
:1033B0003091C001DC01CB0180279127A227B327E0
:1033C0008093BD019093BE01A093BF01B093C00153
:1033D0001F910F910C94E0140895CF92DF92EF9219
:1033E000FF920F931F93CF93DF938C01C090C10185
:1033F000D090C201E090C301F090C4018091BD0162
:103400009091BE01A091BF01B091C001C82AD92AF4
:10341000EA2AFB2ACFE1D0E0D701C6010C2E04C076
:10342000B695A795979587950A94D2F780FF06C021
:10343000B8018C2F0E94B908019721F4219760F7F9
:1034400080E001C08C2FDF91CF911F910F91FF90F1
:10345000EF90DF90CF900895CF93DF93EC010E941F
:10346000ED19BE010E94B908DF91CF910895CB01FB
:103470000E942C1A08958091C501859585958595A2
:1034800008958091C5018770089598E0899F900103
:103490001124262B2093C5010C9431192091C501CC
:1034A000809582238093C501982F977069F430E04E
:1034B000482F552747FD50952417350729F0859546
:1034C000859585950C94521908959091C501977032
:1034D00081E009F480E0089590910C01992321F096
:1034E00090910D01911109C020910E0130910F01B1
:1034F000F90132969FEF40E01FC0982F9695969560
:1035000096959F3050F5E0910E01F0910F01E90F73
:10351000F11D877021E030E0A90102C0440F551F62
:103520008A95E2F7CA019181892B818308959F3F93
:1035300039F04F5F4E3041F051915813F8CF0DC024
:103540005111F7CF942FF5CF9F3F39F0F901E90FD3
:10355000F11D97FDFA9582830895089590910C01CD
:10356000992321F090910D01911109C020910E0134
:1035700030910F01F9013296205F3F4F1FC0982F05
:103580009695969596959F30F0F4E0910E01F09106
:103590000F01E90FF11D877021E030E0A90102C0A1
:1035A000440F551F8A95E2F7CA01809591818923BE
:1035B000818308953196E217F30729F090819813DB
:1035C000F9CF1082F7CF089581E090E0E0910E01ED
:1035D000F0910F01E80FF91F1082019680319105DB
:1035E000A9F708959091D901892B8093D901089565
:1035F00080959091D90189238093D90108951092E3
:10360000D90108959091D801892B8093D80108950C
:1036100080959091D80189238093D80108951092C4
:10362000D80108959091D701892B8093D7010895EF
:1036300080959091D70189238093D70108951092A6
:10364000D70108958093C60108951092C601089588
:1036500080910E0190910F01FC0131969C01205F39
:103660003F4F80E0919191118F5FE217F307D1F7FF
:103670000895E0910E01F0910F018091D9018083AE
:10368000E0910E01F0910F0190818091D801892B7A
:103690008083E0910E01F0910F0190818091D7011C
:1036A000892B80838091C601882361F0E0910E010F
:1036B000F0910F019081892B80830E94281B81113A
:1036C0001092C60180910E0190910F010C94671029
:1036D00020E0009739F0AC01415051098423952333
:1036E0002F5FF7CF822F0895CF92DF92EF92FF9254
:1036F0006C01EE24FF24C114D104E104F10421F093
:10370000C701B60120E101C020E0C72ED82EE92E66
:10371000FF24C114D104E104F10419F0285FC701AA
:10372000B6016B017C0154E0F694E794D794C794FA
:103730005A95D1F7C114D104E104F10419F02C5FBA
:10374000C701B6016B017C0142E0F694E794D7947F
:10375000C7944A95D1F7C114D104E104F10419F0DA
:103760002E5FC701B601DC01CB01B695A7959795F1
:103770008795892B8A2B8B2B09F02F5F822FFF9047
:10378000EF90DF90CF9008958091F101843021F186
:103790001092DB0120E488E190E00FB6F894A89540
:1037A000809360000FBE2093600080E00E94540967
:1037B00083B7817F846083BF83B7816083BF789440
:1037C000889583B78E7F83BF88E10FB6F894809386
:1037D0006000109260000FBE0895089508950E9441
:1037E000ED1B0E94AB030E94EE1B0E94A00491E01F
:1037F000811101C090E0892F08950E94F4140E9465
:103800005B100C94540982E084BD93E095BD9AEF5F
:1038100097BD80936E0008952FB7F8948091DC01D6
:103820009091DD01A091DE01B091DF012FBF0895DD
:10383000CF92DF92EF92FF920F931F932FB7F894DE
:103840004091DC015091DD016091DE017091DF015A
:103850002FBF6A017B01EE24FF248C0120E030E0C1
:10386000C016D106E206F30610F4415051099A0140
:10387000281B390BC9011F910F91FF90EF90DF902A
:10388000CF9008951F920F920FB60F9211248F932D
:103890009F93AF93BF938091DC019091DD01A09144
:1038A000DE01B091DF010196A11DB11D8093DC0105
:1038B0009093DD01A093DE01B093DF01BF91AF9142
:1038C0009F918F910F900FBE0F901F9018950E949F
:1038D000580DF8942FEF87EA91E6215080409040F0
:1038E000E1F700C0000087E090EBDC018093FB0172
:1038F0009093FC01A093FD01B093FE019CE088E150
:103900000FB6F894A895809360000FBE9093600066
:10391000FFCFEF92FF920F931F93CF93DF93D82F98
:10392000CDE08C2F0E94990405E010E0E82EF12CE8
:10393000C701002E02C0959587950A94E2F780FF93
:1039400009C0602F7C2F80E00E946406D81302C05B
:1039500081E006C00150110958F7C15010F780E00E
:10396000DF91CF911F910F91FF90EF900895CF932A
:10397000C82F8CE20E94891C882321F08C2FCF91C4
:103980000C94891C80E0CF910895CF930E940C1E67
:10399000811102C00E94F21DC5E6C15049F00E948B
:1039A000AB038FE39CE90197F1F700C00000F5CF6E
:1039B00089E20E94B71C811113C18AE20E94B71CE0
:1039C00081110E94F21D85E00E94B71C81110E94A6
:1039D000671C0E94171E8093DA0187E00E94B71CC3
:1039E0008823A9F18BE10E94B71C882351F08091B4
:1039F000DA0181FB222720F991E0922790FB81F9DF
:103A00000EC08EE00E94B71C882361F08091DA011D
:103A100082FB222720F991E0922790FB82F9809384
:103A2000DA0115C080E10E94B71C9091DA01882369
:103A300041F093FB222720F981E0822780FB93F954
:103A400004C0892F809580FB90F99093DA018091D2
:103A5000DA010E941B1E0E94291E8093FA0180EE4B
:103A60000E94B71C882341F08091FA01982F90950D
:103A700090FB80F98093FA0189E30E94B71C8823A8
:103A800059F08091FA0181FB222720F991E09227D9
:103A900090FB81F98093FA0182EE0E94B71C882383
:103AA00059F08091FA0182FB222720F991E09227B8
:103AB00090FB82F98093FA0186EE0E94B71C88235E
:103AC00059F08091FA0183FB222720F991E0922797
:103AD00090FB83F98093FA0183EE0E94B71C882340
:103AE00059F08091FA0184FB222720F991E0922776
:103AF00090FB84F98093FA0185E30E94B71C882328
:103B000059F08091FA0185FB222720F991E0922754
:103B100090FB85F98093FA0181E30E94B71C88230A
:103B200059F08091FA0186FB222720F991E0922733
:103B300090FB86F98093FA0181E10E94B71C8823EB
:103B400059F08091FA0187FB222720F991E0922712
:103B500090FB87F98093FA018091FA010E942D1E53
:103B60008091FA0187FB882780F980930D0187E215
:103B70000E94B71CC82F8EE10E94B71C8111C26041
:103B80008FE10E94B71C8111C46080E20E94B71CC3
:103B90008111C86081E20E94B71C8111C06182E27C
:103BA0000E94B71C8111C06283E20E94B71C811180
:103BB000C06484E20E94B71C882311F0C06802C070
:103BC000CC2329F08C2F0E94241E6C2F03C00E944E
:103BD000201E682F70E080E090E0CF910C94B41824
:103BE000CF9108956DEE7EEF80E090E00E945E241C
:103BF00060E082E090E00E944C2460E083E090E08E
:103C00000E944C2460E084E090E00E944C2460E03C
:103C100085E090E00C944C2480E090E00E944624E3
:103C200021E08D3E9E4F09F020E0822F089582E032
:103C300090E00C943E24682F82E090E00C944C2499
:103C400083E090E00C943E24682F83E090E00C9495
:103C50004C2484E090E00C943E24682F84E090E0B3
:103C60000C944C248091E20180FF0BC06091130101
:103C700085E0689FB00111247595679575956795E6
:103C80002BC081FF09C06091130185E0689FB001DE
:103C900011247595679520C082FF07C060911301BC
:103CA00085E0689FB001112417C09091E30199232A
:103CB000D1F060911201961788F72091130185E0E9
:103CC000289F90011124929FA001939F500D1124D1
:103CD00070E0CA010E9410246038710540F461153B
:103CE000710539F002C065E070E0862F08958FE716
:103CF000089581E008958091E20180FF08C06091FD
:103D0000110170E0759567957595679521C081FFE4
:103D100006C06091110170E07595679519C082FF2A
:103D200004C06091110170E010C09091E3019923EB
:103D3000C1F0609110019617A0F780911101899F41
:103D4000C001112470E00E9410246038710528F42D
:103D50006115710521F0862F08958FE7089581E0A0
:103D6000089561E070E0F4CF803F21F40E94321E9C
:103D7000819504C0813F29F40E94321E8093E601A0
:103D80000895823F21F40E94321E819504C0833F32
:103D900029F40E94321E8093E5010895893F19F4A9
:103DA0000E947B1E05C08A3F31F40E947B1E8195D4
:103DB0008093E70108958B3F21F40E947B1E81953B
:103DC00004C08C3F29F40E947B1E8093E801089573
:103DD000843F21F48091E401816017C0853F21F484
:103DE0008091E401826011C0863F21F48091E4015A
:103DF00084600BC0873F21F48091E401886005C096
:103E0000883F31F48091E40180618093E40108955A
:103E10008D3F21F48091E20181600BC08E3F21F43F
:103E20008091E201826005C08F3F29F48091E20118
:103E300084608093E2010895803F39F48091E60127
:103E400087FF6CC01092E60169C0813F29F4809120
:103E5000E6011816BCF362C09091E501823F29F497
:103E600097FF5CC01092E50159C0833F19F4191601
:103E7000CCF354C0893F41F48091E70118160CF04F
:103E80004DC01092E7014AC08A3F29F48091E701B2
:103E900087FF44C0F6CF8B3F39F48091E80187FF5C
:103EA0003DC01092E8013AC08C3F29F48091E801AE
:103EB0001816BCF333C0843F21F48091E4018E7F57
:103EC00017C0853F21F48091E4018D7F11C0863FAA
:103ED00021F48091E4018B7F0BC0873F21F4809116
:103EE000E401877F05C0883F31F48091E4018F7E33
:103EF0008093E40113C08D3F21F48091E2018E7F15
:103F00000BC08E3F21F48091E2018D7F05C08F3F71
:103F100029F48091E2018B7F8093E2018091E50199
:103F200081110EC08091E60181110AC08091E701E4
:103F3000811106C08091E801811102C01092E30155
:103F4000089584EE91E00E9472100E940C1C9093E0
:103F5000E1018093E00108951F93CF93DF93809157
:103F6000E0019091E1010E94181CAC019091E301E5
:103F7000992321F02091140130E006C02091150111
:103F80008AE0289F900111244217530708F486C045
:103F90008091E501C091E601D091E7011091E8011F
:103FA000811107C0C11176C0D11174C0111172C046
:103FB00075C09F3F19F09F5F9093E301181624F49A
:103FC0000E94321E8093E5018091E50187FF05C0C4
:103FD0000E94321E81958093E5011C1624F40E94F4
:103FE000321E8093E6018091E60187FF05C00E94A2
:103FF000321E81958093E6016091E501662339F1D7
:10400000C091E601CC2319F1772767FD7095872FC2
:10401000972F0E94212323E333E343E35FE30E94CE
:1040200085230E94EE226093E5016C2F772767FDC0
:104030007095872F972F0E94212323E333E343E3D7
:104040005FE30E9485230E94EE226093E6011D1625
:1040500024F40E947B1E8093E7018091E70187FF93
:1040600005C00E947B1E81958093E701111624F400
:104070000E947B1E8093E8018091E80187FF05C0C4
:104080000E947B1E81958093E801DF91CF911F9163
:104090000C94A11F9F3F09F08ECF96CFDF91CF9157
:1040A0001F910895E4EEF1E085E0DF011D928A950D
:1040B000E9F71092E3011092E2010895833081F153
:1040C00028F4813059F08230D1F00895853009F418
:1040D00049C0B8F1863009F456C0089580911501A1
:1040E000262F30E0280F311D2F3F310524F4680FB3
:1040F0006093150108958FEF8093150108958091C5
:104100001401262F30E0280F311D2F3F310524F4F4
:10411000680F6093140108958FEF80931401089540
:1041200080911301262F30E0280F311D2F3F3105DC
:1041300024F4680F6093130108958FEF80931301A7
:10414000089580911201262F30E0280F311D2F3F56
:10415000310524F4680F6093120108958FEF809366
:104160001201089580911101262F30E0280F311D92
:104170002F3F310524F4680F6093110108958FEFEC
:1041800080931101089580911001262F30E0280FAF
:10419000311D2F3F310524F4680F609310010895FD
:1041A0008FEF809310010895833011F128F481304E
:1041B00049F0823091F00895853081F120F1863008
:1041C000C1F1089580911501681720F4861B809332
:1041D0001501089510921501089580911401681732
:1041E00020F4861B80931401089510921401089501
:1041F00080911301681720F4861B809313010895A2
:1042000010921301089580911201681720F4861B03
:104210008093120108951092120108958091110166
:10422000681720F4861B80931101089510921101E4
:10423000089580911001681720F4861B8093100167
:1042400008951092100108950F931F938D3109F472
:104250006BC008F03FC08E3009F47FC0C0F48730D7
:1042600009F469C068F4863009F0B1C08091DA01C0
:10427000817F8E7F8093DA0181E08093EA01A8C07C
:10428000883009F4A2C08B3009F49FC0A0C08631E9
:1042900009F49BC078F4803109F472C0813109F0CF
:1042A00096C00E94F41490910D0181E089278093BB
:1042B0000D018BC0893109F488C08B3109F087C0AA
:1042C0008091DA0181FB222720F991E0922790FB6F
:1042D00081F94CC0853309F470C048F4873209F481
:1042E0006CC008F459C0893209F467C070C08334C7
:1042F00038F48A3308F04EC0883309F466C067C0CA
:10430000833409F45AC0883409F061C00E94F4145F
:104310000FEF13ED20E3015010402040E1F700C003
:1043200000000E94671C51C00E94A8220E945B10DE
:104330000E9454094AC09091DA01892F80958170BA
:1043400080FB90F929F0966098609093DA0140C064
:10435000997F977F9093DA0138C08091DA0182FBD0
:10436000222720F991E0922790FB82F98093DA01CD
:10437000992359F18091DA0181608093DA0125C097
:104380008091DA0183FB222720F991E0922790FBAC
:1043900083F9ECCF895301C08D5141E050E060E0DA
:1043A00070E08A019B0104C0000F111F221F331F00
:1043B0008A95D2F7C901B80104C061E070E080E0DD
:1043C00090E00E94B4180E94F41481E001C080E0E3
:1043D0001F910F91089580E0089580E00895CF9394
:1043E000C82F8091EA01813079F018F08230E9F12C
:1043F00087C0E0910E01F0910F018081813169F059
:10440000823209F07FC009C0E0910E01F0910F01E6
:104410008081813111F0823261F48C2F0E94EB2176
:10442000811104C08C2F0E9424211DC081E090E0E6
:104430001AC08C2F0E94ED21811114C0C43179F073
:1044400048F4CB3079F0C03109F060C082E080934D
:10445000EA0108C0C93219F0C83321F057C01092E0
:10446000EA0154C081E0817053C0C93289F118F566
:10447000C43171F1A8F4C73009F046C08AE08093D6
:10448000150194E19093140193E0909313018093AC
:10449000120188E08093110188E28093100134C0FA
:1044A000CE51C63088F5EC2FF0E0E65DFE4F8081FE
:1044B0008093E90129C0CE34E9F020F4CB3421F512
:1044C0006AE013C0C13579F0C235F1F461E00DC086
:1044D0008091E901882319F01092E90115C081E06B
:1044E0008093EA0115C061E006C08091E9010E9455
:1044F0005E200AC06AE08091E9010E94D42004C0D5
:104500001092EA0180E004C081E002C080E0ABCFFD
:10451000CF910895E1E8F0E0808188608083808118
:10452000816080838FB7F89493E09093890090ED39
:10453000909388008FBF0895EFE6F0E0808182605D
:1045400080830895EFE6F0E080818D7F8083089579
:10455000EFE6F0E0908182E08927808308951F9242
:104560000F920FB60F9211242F933F934F935F93A7
:104570006F937F938F939F93AF93BF93EF93FF932B
:104580008091EB019091EC0101969093EC01809366
:10459000EB01811103C082E00E945409E091EC011B
:1045A000E695E695F0E0ED58FA4FE4918091EB0145
:1045B0008E1303C080E00E945409FF91EF91BF91D8
:1045C000AF919F918F917F916F915F914F913F91AB
:1045D0002F910F900FBE0F901F90189504D06894E4
:1045E000B1118DC0089570D088F09F5790F0B92F09
:1045F0009927B751A0F0D1F0660F771F881F991F38
:104600001AF0BA95C9F712C0B13081F077D0B1E095
:10461000089574C0672F782F8827B85F39F0B93FA5
:10462000CCF3869577956795B395D9F73EF4909539
:104630008095709561957F4F8F4F9F4F0895E894B7
:1046400009C097FB3EF490958095709561957F4FDA
:104650008F4F9F4F9923A9F0F92F96E9BB27939588
:10466000F695879577956795B795F111F8CFFAF498
:10467000BB0F11F460FF1BC06F5F7F4F8F4F9F4FC9
:1046800016C0882311F096E911C0772321F09EE827
:10469000872F762F05C0662371F096E8862F70E08D
:1046A00060E02AF09A95660F771F881FDAF7880F67
:1046B0009695879597F9089557FD9058440F551F83
:1046C00059F05F3F71F04795880F97FB991F61F094
:1046D0009F3F79F087950895121613061406551F0B
:1046E000F2CF4695F1DF08C0161617061806991F77
:1046F000F1CF86957105610508940895E894BB276C
:1047000066277727CB0197F908950BD078C069D039
:1047100028F06ED018F0952309F05AC05FC011241C
:10472000EECFCADFA0F3959FD1F3950F50E0551F50
:10473000629FF001729FBB27F00DB11D639FAA27F6
:10474000F00DB11DAA1F649F6627B00DA11D661F45
:10475000829F2227B00DA11D621F739FB00DA11D66
:10476000621F839FA00D611D221F749F3327A00D20
:10477000611D231F849F600D211D822F762F6A2FBC
:1047800011249F5750408AF0E1F088234AF0EE0F41
:10479000FF1FBB1F661F771F881F91505040A9F74E
:1047A0009E3F510570F014C0AACF5F3FECF3983ED6
:1047B000DCF3869577956795B795F795E7959F5FB5
:1047C000C1F7FE2B880F911D9695879597F908954F
:1047D00097F99F6780E870E060E008959FEF80ECB4
:1047E000089500240A941616170618060906089557
:1047F00000240A9412161306140605060895092EBD
:104800000394000C11F4882352F0BB0F40F4BF2B2B
:1048100011F460FF04C06F5F7F4F8F4F9F4F08956B
:1048200097FB072E16F4009407D077FD09D00E945D
:104830002A2407FC05D03EF4909581959F4F08955A
:10484000709561957F4F0895EE0FFF1F0590F491CD
:10485000E02D0994AA1BBB1B51E107C0AA1FBB1F77
:10486000A617B70710F0A61BB70B881F991F5A95FC
:10487000A9F780959095BC01CD010895F999FECFD7
:1048800092BD81BDF89A992780B50895A8E1B0E05E
:1048900042E050E00C946624262FF999FECF92BD99
:1048A00081BDF89A019700B4021639F01FBA20BDF5
:1048B0000FB6F894FA9AF99A0FBE08950196272F29
:1048C0000E944D240C944C24DC01CB01FC01F9998D
:1048D000FECF06C0F2BDE1BDF89A319600B40D924C
:0C48E00041505040B8F70895F894FFCF05
:1048EC0002205609E409C1098D0959090101C701C2
:1048FC0028080A03140A3F4D36393405E704B1047D
:10490C0078040B0424043D04560401020304050638
:04491C00070809007F
:00000001FF
